:1000000000308A0004280000FF238316900000308F
:100010008A001F283408A10133020318122833086C
:10002000A0001E28A0010830B500B30DA00D3408B3
:1000300020020318A000A10DB50B1528003484017F
:100040001F30830583161F08F0399F0083121F138A
:1000500007309F00A5010130A600A701A801A90152
:100060002A14AB010730990083160508831219087A
:100070008C1183161F080F399F0083121F080C393B
:100080009F000130831695008113FF308500831295
:100090000508AD0083169B019C131C141A088312DB
:1000A000B200B3000A30B4000A202008AC00831666
:1000B000851083128514B001AF013008073C031C82
:1000C0007428031D67282F08CF3C031C7428AE0139
:1000D0002E0F6B286F2800000130AE076828013012
:1000E000AF070318B00A5D280130AA062A187A283B
:1000F00005127B280516831605128312AE012E0801
:100100003F3C031C9F288316851083128510AD0188
:100110002C082D0203188F280130AD07882883167C
:10012000851083128514AD012C08093C2D0203189B
:100130009C280130AD0794280130AE077F280310BA
:100140002B0DB10083160514003083120518013001
:100150003104AB002B08803C031DCE2801302C0756
:10016000B200B3000A30B4000A202008AC008316A5
:100170009B0183122C0883169A001C1583120B080E
:10018000A0008B13831655309D00AA309D009C144F
:100190009C18C8281C11831220088B047428630043
:02400E00C401EB
:00000001FF
